:03004300020900AF
:030053000209009F
:10090000020DD200020E1800020E0200020DEA00D3
:10091000020C04000208BE000200320002004A007D
:10092000020052000208FB000208FC000208FD0061
:100930000208FE000208FF00020E7D00020E7E008B
:10094000020E7F0002004A00020E8000020E8100AB
:10095000020E8200020E8300020E8400020E850049
:10096000020E860002004A0002004A0002004A000D
:10097000020E8700020E8800020E8900020E8A0015
:10098000020E8B00020E8C00020E8D00020E8E00F5
:10099000020E8F00020E9000020E9100020E9200D5
:1009A000020E9300020E9400020E9500020E9600B5
:0809B000020B9000020E9700FB
:100800001201000200000040E4E441110000010276
:1008100003010A06000200000040010009022E0048
:1008200001010080320904000004FF0000000705F8
:10083000020200020007050402000200070586020A
:100840000002000705880200020009022E000101D3
:100850000080320904000004FF00000007050202C6
:100860004000000705040240000007058602400022
:10087000000705880240000004030904180358001B
:100880006F00720063006F006D0020004C00740068
:1008900064002E0028035800500044002000280067
:1008A00020004200610073006500640020006F00BA
:0E08B0006E002000580050005000290000008B
:100C3A001201000200000040E4E442110000010237
:100C4A0000011201000200000040E4E4401100002B
:100C5A0001020001000102030405060708090A0B44
:040C6A000C0D0E0F50
:080E5C004100100041001100EB
:1009B80090E600E054E74410F000000090E604746C
:1009C80080F00000007406F0000000E4F000000071
:1009D80090E6107420F000000090E611F00000008E
:1009E80090E61274A2F000000090E61374A0F000E4
:1009F800000090E61474E2F000000090E61574E040
:100A0800F000000090E6047480F00000007404F028
:100A1800000000E4F000000090E6497482F0000055
:100A280000F000000090E6187410F000000090E656
:100A38001A7408F000000090E619E054FEF0000077
:100A48000090E61BE054FEF000000090E6917480F0
:100A5800F0000000F000000090E695F0000000F0C3
:070A680000000043AF012272
:1005960078007C007D017BFF7A0C795E7E007F10FF
:1005A6001204F0C205E5AA30E2030206F1E5AA301C
:1005B600E7030206F175310075320490F400E02479
:1005C600FE700302067124FA700302068D24F87089
:1005D600030206B624F070030206C0241F6003025D
:1005E60006CA90FC007401F090F401E090FC01F062
:1005F60090F402E090FC02F0D2B690F401E0701A9A
:10060600A3E0701630B01374C0120D78C2B67F081E
:10061600120D7ED2B67F08120D7E30B04690E6945B
:10062600E0FE90E695E07C002400FFEC3ECF24FC43
:10063600CF34FFFE7B017AF47904120AFB501C903A
:10064600FC0330B4117408F07FD07E07120D80745D
:1006560003120D78807A7404F0807590FC0374029E
:10066600F0806D90FC037401F0806590FC007402CC
:10067600F0E4A3F0A3F030B406A37410F080069063
:10068600FC037420F0804975310075321190FC002E
:100696007408F07A007B007D017F50120DB67F5002
:1006A600120BCC7AFC7B017D107F50120D9A8020B4
:1006B600750A0C750B3AD2028028750A0C750B4C1C
:1006C600D202801E75310075320190FC0074AAF0CA
:1006D600E53190E69CF0000000E53290E69DF000E2
:0B06E600000090E6957480F00000001A
:0106F10022E6
:0C0D780090E601F07F147E007D007C00FE
:100D84008F368E358D348C33783374FF120578ECBE
:060D94004D4E4F70F322EA
:0A0AFB008E338F348B358A3689372D
:100B0500E4F538F539C3E5399534E538953350338F
:100B1500AB35AA36A937853982853883120516FF84
:100B2500E4FEC2B2EF1392B7EFC313FFD2B20EBE0B
:100B350008F0C2B220B002C3220539E53970C605F6
:040B45003880C2D35F
:010B49002289
:02004100D322C8
:02004E00D322BB
:02005000D322B9
:080E650090E6BAE0F51DD3226E
:100E2E0090E740E51DF0E490E68AF090E68B04F042
:020E3E00D322BD
:080E6D0090E6BAE0F51CD32267
:100E400090E740E51CF0E490E68AF090E68B04F031
:020E5000D322AB
:0207FA00D32208
:0207FC00D32206
:0207FE00D32204
:100D2B0090E6B9E0242F600D04701990E604E0FF03
:100D3B00430780800890E604E0FF53077F00000024
:070D4B00EFF08002D322C388
:010D5200227E
:100DD200C0E0C083C082D2015391EF90E65D7401FE
:080DE200F0D082D083D0E03292
:100E0200C0E0C083C0825391EF90E65D7404F0D0DD
:060E120082D083D0E03223
:100E1800C0E0C083C0825391EF90E65D7402F0D0C9
:060E280082D083D0E0320D
:100C0400C0E0C083C08285100C85110D850D8285DE
:100C14000C83A37402F085080E85090F850F828565
:100C24000E83A37407F05391EF90E65D7410F0D037
:060C340082D083D0E03203
:100DEA00C0E0C083C082D2045391EF90E65D7408DC
:080DFA00F0D082D083D0E0327A
:1008BE00C0E0C083C08290E680E030E72085080C5F
:1008CE0085090D850D82850C83A37402F085100EAB
:1008DE0085110F850F82850E83A37407F05391EF58
:0D08EE0090E65D7420F0D082D083D0E0321F
:01003200329B
:01004A003283
:01005200327B
:0108FB0032CA
:0108FC0032C9
:0108FD0032C8
:0108FE0032C7
:0108FF0032C6
:010E7D003242
:010E7E003241
:010E7F003240
:010E8000323F
:010E8100323E
:010E8200323D
:010E8300323C
:010E8400323B
:010E8500323A
:010E86003239
:010E87003238
:010E88003237
:010E89003236
:010E8A003235
:010E8B003234
:010E8C003233
:010E8D003232
:010E8E003231
:010E8F003230
:010E9000322F
:010E9100322E
:010E9200322D
:010E9300322C
:010E9400322B
:010E9500322A
:010E96003229
:100B9000C0E0C083C08290E6D1E0900010F090E603
:100BA000D0E4F000000090E6D17402F000000053A1
:100BB00091BF00000090E66104F000000090E6990B
:0C0BC00004F075BB06D082D083D0E03278
:010E97003228
:0A0E52000001020203030404050579
:10028D00E4F52CF52BF52AF529C204C200C203C2F0
:10029D0001C202D2B675B5C4D2B61209B8120E7526
:1002AD007E087F008E0A8F0B751208751312750864
:1002BD000875091C75100875114A7514087515789F
:1002CD00EE54C0700302039A752D00752E808E2F8B
:1002DD008F30C374BC9FFF74089ECF2402CF3400AF
:1002ED00FEE48F288E27F526F525F524F523F52236
:1002FD00F521AF28AE27AD26AC25AB24AA23A92224
:10030D00A821C31205655033E5302524F582E52F6C
:10031D003523F583E0FFE52E2524F582E52D3523E4
:10032D00F583EFF0E5242401F524E43523F523E4EA
:10033D003522F522E43521F52180B7852D0A852E4C
:10034D000B74002480FF740834FFFEC3E5139FF582
:10035D0013E5129EF512C3E50D9FF50DE50C9EF507
:10036D000CC3E50F9FF50FE50E9EF50EC3E5099F36
:10037D00F509E5089EF508C3E5119FF511E5109EF9
:10038D00F510C3E5159FF515E5149EF514D2E84358
:10039D00D82090E668E0440BF090E65CE0443DF038
:1003AD00000000E4F5A2000000D2AFD20512000358
:1003BD0090E680E054F7F0538EF8C20412059630A3
:1003CD00021B90E680E054FDF0E054F7F0D20512E8
:1003DD00000390E680E04402F0C204C20230010541
:1003ED00120056C2013004D412004150CFC2041283
:1003FD000D5320001690E682E030E704E020E1EF97
:10040D0090E682E030E604E020E0E4120CD4120025
:03041D004E80A965
:0B00360090E50DE030E402C322D3226D
:1000560090E6B9E0700302011514700302019224C0
:10006600FE700302021524FB700302010F147003D5
:100076000201091470030200FD1470030201032437
:10008600056003020279120050400302028590E6E1
:10009600BBE024FE602714603824FD60111460273D
:1000A60024067050E50A90E6B3F0E50B803C12009A
:1000B60036503EE51290E6B3F0E513802DE50C9040
:1000C600E6B3F0E50D8023E50E90E6B3F0E50F808C
:1000D6001990E6BAE0FF120D00AA06A9077B01EA0D
:1000E600494B600DEE90E6B3F0EF90E6B4F00202F5
:1000F60085020274020274120E40020285120E6D0F
:10010600020285120E65020285120E2E0202851269
:1001160007FA400302028590E6B8E0247F601514D2
:10012600601924027063A200E43325E0FFA203E411
:10013600334F8041E490E740F0803F90E6BCE054C6
:100146007EFF7E00E0D394807C0040047D01800227
:100156007D00EC4EFEED4F2452F582740E3EF58383
:10016600E493FF3395E0FEEF24A1FFEE34E68F82A1
:10017600F583E0540190E740F0E4A3F090E68AF0BE
:1001860090E68B7402F00202850202741207FC40AC
:100196000302028590E6B8E024FE6016240260039E
:1001A60002028590E6BAE0B40105C20002028502A9
:1001B600027490E6BAE0705590E6BCE0547EFF7E8D
:1001C60000E0D394807C0040047D0180027D00EC39
:1001D6004EFEED4F2452F582740E3EF583E493FFF6
:1001E6003395E0FEEF24A1FFEE34E68F82F583E03F
:1001F60054FEF090E6BCE05480131313541FFFE046
:10020600540F2F90E683F0E04420F08072805F1256
:1002160007FE506B90E6B8E024FE60192402704E8B
:1002260090E6BAE0B40104D200805490E6BAE064E5
:1002360002604C803990E6BCE0547EFF7E00E0D33D
:1002460094807C0040047D0180027D00EC4EFEED32
:100256004F2452F582740E3EF583E493FF3395E006
:10026600FEEF24A1FFEE34E68F82F583800D90E643
:10027600A08008120D2B500790E6A0E04401F090F4
:06028600E6A0E04480F058
:01028C00224F
:0300330002004682
:0400460053D8EF326A
:100CD40090E682E030E004E020E60B90E682E0302B
:100CE400E119E030E71590E680E04401F07F147EDE
:0C0CF40000120B4A90E680E054FEF02253
:1000030030050990E680E0440AF0800790E680E03E
:100013004408F07FDC7E05120B4A90E65D74FFF026
:0F00230090E65FF05391EF90E680E054F7F02203
:080E7500E4F51BD2E9D2AF2223
:100BCC00AD0790E678E020E6F9C2E990E678E044DB
:100BDC0080F0ED25E090E679F090E678E030E0F9F1
:100BEC0090E678E04440F090E678E020E6F990E674
:080BFC0078E030E1D6D2E922D5
:100CA200AC0790E678E020E6F9E51B702390E67841
:100CB200E04480F0EC25E090E679F08D16AF03A9D0
:100CC200077517018A188919E4F51A751B01D322D1
:020CD200C3223B
:100C6E00AC0790E678E020E6F9E51B702590E67873
:100C7E00E04480F0EC25E0440190E679F08D16AF6B
:100C8E0003A9077517018A188919E4F51A751B034C
:040C9E00D322C32278
:03004B000206F2B8
:1006F200C0E0C083C082C085C084C086758600C049
:10070200D075D000C000C001C002C003C006C0073F
:1007120090E678E030E206751B060207DC90E67888
:10072200E020E10CE51B64026006751B070207DC92
:10073200E51B24FE605F14603624FE70030207CDC1
:1007420024FC70030207D9240860030207DCAB17FC
:10075200AA18A919AF1A051A8F82758300120516F5
:1007620090E679F0E51A65167070751B05806B903E
:10077200E679E0AB17AA18A919AE1A8E8275830022
:10078200120543751B02E5166401704E90E678E08F
:100792004420F08045E51624FEB51A0790E678E07D
:1007A2004420F0E51614B51A0A90E678E04440F0C9
:1007B200751B0090E679E0AB17AA18A919AE1A8E3C
:1007C20082758300120543051A800F90E678E04493
:1007D20040F0751B008003751B005391DFD007D0DA
:1007E20006D003D002D001D000D0D0D086D084D0A1
:0807F20085D082D083D0E032F3
:020D0000A90741
:100D0200AE14AF158F828E83A3E064037017AD011A
:100D120019ED7001228F828E83E07C002FFDEC3E64
:080D2200FEAF0580DFE4FEFFD7
:010D2A0022A6
:100D9A00120C6EE51B24FA600E146006240770F329
:0C0DAA00D322E4F51BD322E4F51BD32276
:100DB600120CA2E51B24FA600E146006240770F3D9
:0C0DC600D322E4F51BD322E4F51BD3225A
:100D530090E682E044C0F090E681F0438701000012
:040D6300000000226A
:100B4A008E318F3290E600E054187012E53224019B
:100B5A00FFE43531C313F531EF13F532801590E612
:100B6A0000E05418FFBF100BE53225E0F532E531FD
:100B7A0033F531E5321532AE31700215314E60056A
:060B8A00120D6780EE224F
:100D67007400F58690FDA57C05A3E582458370F99F
:010D77002259
:03000000020A6F82
:0C0A6F00787FE4F6D8FD758139020AB6E4
:10042000E709F608DFFA8046E709F208DFFA803EBE
:1004300088828C83E709F0A3DFFA8032E309F608AB
:10044000DFFA8078E309F208DFFA807088828C8313
:10045000E309F0A3DFFA806489828A83E0A3F608C7
:10046000DFFA805889828A83E0A3F208DFFA804CA1
:1004700080D280FA80C680D4806980F28033801078
:1004800080A680EA809A80A880DA80E280CA8033E1
:1004900089828A83ECFAE493A3C8C582C8CCC58359
:1004A000CCF0A3C8C582C8CCC583CCDFE9DEE78029
:1004B0000D89828A83E493A3F608DFF9ECFAA9F0A8
:1004C000EDFB2289828A83ECFAE0A3C8C582C8CCFE
:1004D000C583CCF0A3C8C582C8CCC583CCDFEADE17
:1004E000E880DB89828A83E493A3F208DFF980CC79
:1004F00088F0EF60010E4E60C388F0ED2402B40472
:100500000050B9F582EB2402B4040050AF23234518
:06051000822390047073C9
:10051600BB010CE58229F582E5833AF583E022509A
:1005260006E92582F8E622BBFE06E92582F8E222E4
:0D053600E58229F582E5833AF583E49322FE
:10054300F8BB010DE58229F582E5833AF583E8F0EE
:10055300225006E92582C8F622BBFE05E92582C89A
:02056300F22282
:10056500EB9FF5F0EA9E42F0E99D42F0E89C45F0EC
:010575002263
:100576007401FF3395E0FEFDFC080808E6CF2FF670
:1005860018E6CE3EF618E6CD3DF618E6CC3CF62249
:100A7B0002028DE493A3F8E493A34003F68001F202
:100A8B0008DFF48029E493A3F85407240CC8C3337C
:100A9B00C4540F4420C8834004F456800146F6DF4B
:100AAB00E4800B0102040810204080900E5CE47E71
:100ABB00019360BCA3FF543F30E509541FFEE49340
:100ACB00A360010ECF54C025E060A840B8E493A307
:100ADB00FAE493A3F8E493A3C8C582C8CAC583CA32
:100AEB00F0A3C8C582C8CAC583CADFE9DEE780BEEA
:010E6400008D
:00000001FF
